:100000000C942A000C9447000C9447000C94470071
:100010000C9447000C94F3060C9447000C94A00633
:100020000C9447000C9447000C9437060C9447003E
:100030000C9447000C945C010C94CB010C940802C6
:100040000C9447000C9447000C9447000C94470014
:100050000C94470011241FBECFE5D8E0DEBFCDBF12
:1000600010E0A0E6B0E0ECEBFEE002C005900D92DF
:10007000AC36B107D9F721E0ACE6B0E001C01D9283
:10008000A638B207E1F70E94A3050C945C070C9414
:10009000000080917B0020917A0090E0922B909359
:1000A0006E0080936D0080917900863079F08091A8
:1000B0007900853059F080917D0020917C0090E09E
:1000C000922B9093700080936F00089581E090E0F0
:1000D0009093700080936F00089520916D0030918F
:1000E0006E008217930780F040916D0050916E0072
:1000F00020916F0030917000420F531F21E0841750
:10010000950710F4822F089520E0822F08958091A2
:100110007500089580936C000895CF93DF93EC01F0
:100120006F5F09F43EC0FC01A62FB0E0BC016A0F6E
:100130007B1F2FEF3FEF9081292798E0A9014170A5
:10014000552736952795452B21F081E0282780EA11
:100150003827915099F73196E617F70761F7A9010B
:100160005527632F7727FE01EA0FFB1F808190E060
:100170004817590749F01196AC0FBD1F20836C93A7
:1001800080E0DF91CF910895AD014F5F5F4FDE01B9
:10019000A40FB51F8C9190E08617970779F781E03F
:1001A000F0CF6FEF70E04FEF50E02FEF3FEFA0E0A8
:1001B000B0E0D9CFFB01F695E795F695E795F69572
:1001C000E795E80FF91F808190E06770772702C0FC
:1001D000959587956A95E2F7F901F695E795F69575
:1001E000E795F695E795E40FF51F408127703327D3
:1001F00080FD0AC081E090E001C0880F2A95EAF7EF
:10020000809584238083089581E090E001C0880F69
:100210002A95EAF7842B808308958091750085FFE5
:1002200019C08091730090917400019690937400AE
:10023000809373008091750081FF0DC080917300E1
:1002400090917400079709F1809173009091740068
:10025000429769F0089580917300909174004097DF
:10026000C9F7809175008160809375000895909121
:10027000780080916C00981771F080E2809375008F
:10028000109274001092730008958091750080643C
:1002900080937500089560917100709172006350B1
:1002A00088E790E00E948D00882339F30E9449007E
:1002B00088E08093750008951F920F920FB60F92F9
:1002C00011242F933F938F939F93EF93FF939CB1B0
:1002D00010927400109273008091750083FD04C029
:1002E0008091750084FF2AC08091750083FD1BC03A
:1002F0008091750084FD17C08091750082FD13C048
:100300008091750081FD0FC08091750080FF0BC04A
:100310009093780082E28093750081E090E0909362
:10032000720080937100FF91EF919F918F913F91A7
:100330002F910F900FBE0F901F9018958091750010
:1003400082FDD2CF8091750081FFCECF8091750064
:1003500080FDCACF20917100309172002F3F31058E
:1003600049F040F080E28093750010927400109282
:100370007300D9CFE0917100F0917200E858FF4FFF
:100380009083809171009091720001969093720019
:1003900080937100C8CF1F920F920FB60F92112455
:1003A0002F933F938F939F93EF93FF9380917500CB
:1003B0008F7E8093750080917500846080937500B6
:1003C000E0917100F0917200E858FF4F80818CB984
:1003D00080917100909172000196909372008093C9
:1003E000710080916000209171003091720090E066
:1003F00001968217930709F45598FF91EF919F9109
:100400008F913F912F910F900FBE0F901F901895D5
:100410001F920F920FB60F9211248F93DE9880E2F5
:100420008093750010927400109273008F910F905A
:100430000FBE0F901F90189510BC83E389B982E01E
:100440008BB986E880BD88ED8AB9D69ADE9880E2BD
:1004500080937500089592E0980F90936000682F44
:1004600088E790E00E948D00809175008061809304
:1004700075001092720010927100DE9A559A809168
:100480007500877F809375000895E8E7F0E091811B
:1004900090689183828382E00C942B02CF93DF9348
:1004A00020916D0030916E002617370778F1E091AA
:1004B0006F00F091700020916D0030916E00460F3A
:1004C000571F2E0F3F1F4217530700F1209179004D
:1004D000233059F120917900243039F120917900AD
:1004E000203139F020917900263009F459C080E09C
:1004F00019C040917E0020916F003091700050E053
:10050000220F331F4217530708F065C0809179000E
:1005100080688093790083E080937A0082E00E9473
:100520002B0280E0DF91CF91089520916F003091F0
:100530007000220F331F2C3F310540F720916F00D0
:1005400030917000220F20937A0020916F0030913B
:100550007000422F20916D0030916E00261B370BEA
:10056000220F331F442399F0DC01A20FB31FECE7E5
:10057000F0E080E0EF0121972D913C9111973883B5
:100580002D913D9120838F5F32964813F3CF809158
:100590007A008E5F0E942B0281E0DF91CF91089557
:1005A000A0916D00B0916E00A61BB70BAA0FBB1FE8
:1005B000A80FB91F80917C0020917D0090E0982FBA
:1005C0008827820F911D11969C938E9385E00E943F
:1005D0002B0281E0A7CF40917100509172002091D1
:1005E0007E004950510930E04217530708F48ECF7E
:1005F00020916F0030917000422FA0916D00B0915A
:100600006E00A61BB70BAA0FBB1F2223F9F2E0E86E
:10061000F0E0A80FB91F90E0EF01219728818081B9
:1006200030E0322F2227280F311D11963C932E9354
:1006300012969F5F32964913EFCFC8CFEF92FF9289
:100640000F931F93CF93DF937C018B0180916D00FB
:1006500090916E0086179707C8F120916F00309136
:10066000700080916D0090916E00460F571F820FB1
:10067000931F4817590750F1809179008230C9F1D2
:10068000809179008130A9F1809179008F3069F0F3
:1006900080917900853009F4B5C080E0DF91CF9179
:1006A0001F910F91FF90EF90089580917E0020910F
:1006B0006F003091700090E0880F991F880F991F8C
:1006C000880F991F8217930708F06CC080917900FA
:1006D00080688093790083E080937A0082E00E94B2
:1006E0002B0280E0DF91CF911F910F91FF90EF904F
:1006F000089580916F0090917000893D974030F788
:1007000080916F009091700096958795969587954A
:100710009695879580937A0080916F0090917000F4
:1007200087709927892B99F0E0916F00F091700004
:10073000F695E795F695E795F695E795FF27E55841
:10074000FF4F108280917A008F5F80937A008091B2
:100750006F0090917000892BC1F0C0E0D0E06091F3
:100760006D0070916E00601B710B6C0F7D1F9E0100
:100770004BE750E0C7010E94DA00219680916F009C
:1007800090917000C817D90750F380917A008E5F5E
:100790000E942B0281E0DF91CF911F910F91FF907A
:1007A000EF900895209171003091720080917E0049
:1007B0002950310990E02817390708F487CF809134
:1007C0006F0090917000892BC1F0C0E0D0E02091C3
:1007D0006D0030916E00201B310B2C0F3D1FA701C7
:1007E000BE018FE790E00E94DA00219680916F00B1
:1007F00090917000C817D90750F385E00E942B0232
:1008000081E070CF20916D0030916E00261B370B78
:10081000A70160E070E08CE790E00E94DA00EDCF85
:100820004F925F926F927F928F929F92AF92BF9200
:10083000CF92DF92EF92FF9280917C0190917D01A7
:1008400060E17EE00E941707E62F20917C01309145
:100850007D01A9E8B8E80E944D07AC01569547957F
:10086000529542954F7045275F7045279A010E9427
:100870004D074C0196948794929482946FE086225F
:10088000892496228924FCE3F89DC001F99D900DEE
:1008900011244A01881A990AC0907C01D0907D01E8
:1008A000EE2309F483C0A12CB12C4E2E512C612CC7
:1008B000712C3AE0C32ED12CE12CF12CC301B201F2
:1008C000A70196010E942B07DA01C901880F991F21
:1008D000AA1FBB1F820F931FA41FB51F880F991F4C
:1008E000AA1FBB1F480E591E6A1E7B1E542C44248F
:1008F000C501B401A70196010E942B0769017A0185
:10090000CC0CDD1CEE1CFF1CD701C601820F931F0F
:10091000A41FB51F880F991FAA1FBB1F880D991D03
:10092000AA1DBB1D9201282B392B309385012093E2
:100930008401F901EF70FF27EF59FF4F8081809309
:100940007801F901E07FFF27F295E295EF70EF273C
:10095000FF70EF27EF59FF4F808180937901F901F4
:10096000EE27FF70EF2FFF27EF59FF4F8081809315
:100970007A01C9018827907F892B09F471C0F90198
:10098000EF2FFF27E295EF70EF59FF4F80818093A3
:100990007B01FF90EF90DF90CF90BF90AF909F9042
:1009A0008F907F906F905F904F9008959601A9E887
:1009B000B8E80E944D0796958795929582958F701D
:1009C00089279F708927F89F9001F99F300D112486
:1009D000C21AD30AE12CF12C2401612C712C6AE09B
:1009E000862E912CA12CB12CC301B201A50194013A
:1009F0000E942B07DA01C901880F991FAA1FBB1F8C
:100A0000820F931FA41FB51F880F991FAA1FBB1F1A
:100A1000480E591E6A1E7B1E542C4424C701B60181
:100A2000A50194010E942B0749015A01880C991CC9
:100A3000AA1CBB1CD501C401820F931FA41FB51FA4
:100A4000880F991FAA1FBB1F8C0D9D1DAE1DBF1DBA
:100A50009201282B392B309385012093840169CF93
:100A600080E095CFCF930E94870083FF34C08091B0
:100A700079008530E1F188F58130D1F0833099F546
:100A800089B38F7090E090937F0180937E01809175
:100A9000840190918501909381018093800144E0CD
:100AA00050E060E070E08CE791E0CF910C944E0252
:100AB00048E050E060E070E087E790E00E941E03AD
:100AC00083E090E00E946D00882329F080917700F8
:100AD000877F80937700CF9108958F3041F08031E8
:100AE000F9F08630E9F081E0CF910C944502C09195
:100AF000770048E050E060E070E087E790E00E9417
:100B00001E03C0FD04C08091770080FD14C0809159
:100B1000770081FFE0CFDF9A88EC80937600DBCF0F
:100B200041E050E060E070E08CE791E00E944E020E
:100B3000CF910C9410040E94100480917700816082
:100B400080937700E4CF87B38F6087BBBC9A8CEF2C
:100B500081BB8AB380638ABB8EEF84BBD79A8BB389
:100B600087608BBB88E10E948A000E941C0288E09B
:100B700083BF83E083BF89EF8CBF89B7826089BF61
:100B80008EB58C608EBD84E294EF9BBD8ABD89B723
:100B9000806189BF85B5826085BD89B7806489BF62
:100BA000809177008460809377008CEF93E090933E
:100BB0007D0180937C017894C9B3D1E00CEF13E000
:100BC0000E943205CA9B23C0C99906C080917C014E
:100BD00090917D01069768F5C89914C0C0FF12C0B6
:100BE0008091770080FF37C0809177008D278093B8
:100BF00077009FEF21EE84E0915020408040E1F7A4
:100C000000C00000C9B30E943205CA99DDCF8091AF
:100C10007C0190917D01059690937D0180937C01EC
:100C20000E9410048FE39CE90197F1F700C00000D7
:100C3000CBCF80917C0190917D01059790937D01B0
:100C400080937C010E9410048FE39CE90197F1F7E7
:100C500000C00000C1CF809177008E7F8093770025
:100C600010937D0100937C010E941004BDCF1F9260
:100C70000F920FB60F9211242F933F938F939F9350
:100C80008091770080FF33C0C49AC09B42C088B374
:100C9000807F8A6088BB80917B01982F9C7F92BB6C
:100CA0002BB3837030E1839FC0011124922F9F7C6E
:100CB000892B8BBB8091790185BB80917600811156
:100CC0001EC080917600811109C0DF988091770065
:100CD0008D7F809377008FEF809376009F918F9127
:100CE0003F912F910F900FBE0F901F901895C498B1
:100CF00088B3807F88BB80917600882311F3809130
:100D000076008F3FF1F280917600815080937600DB
:100D1000E5CF88B3807F856088BB80917A01982F6A
:100D20009C7F92BB2BB3837030E1839FC001112461
:100D3000922F9F7C892B8BBB8091780185BBDBCF69
:100D40001F920F920FB60F9211242F933F934F9340
:100D50005F936F937F938F939F93AF93BF93EF9323
:100D6000FF938091770080FD32C080917C0190914B
:100D70007D01892B89F0FF91EF91BF91AF919F91F8
:100D80008F917F916F915F914F913F912F910F9034
:100D90000FBE0F901F901895809177008E7F8093E3
:100DA00077008CEF93E090937D0180937C010E940B
:100DB00010048091770082FFDECFDF9A88EC809369
:100DC000760080917700886080937700D4CF8091FF
:100DD0007C0190917D01019790937D0180937C012E
:100DE0000E941004C2CF1F920F920FB60F921124CF
:100DF0002F933F934F935F936F937F938F939F9323
:100E0000AF93BF93EF93FF930E940D01FF91EF917A
:100E1000BF91AF919F918F917F916F915F914F9112
:100E20003F912F910F900FBE0F901F901895AA1B06
:100E3000BB1B51E107C0AA1FBB1FA617B70710F0C5
:100E4000A61BB70B881F991F5A95A9F780959095F7
:100E5000BC01CD010895A1E21A2EAA1BBB1BFD0106
:100E60000DC0AA1FBB1FEE1FFF1FA217B307E40789
:100E7000F50720F0A21BB30BE40BF50B661F771FE1
:100E8000881F991F1A9469F76095709580959095C1
:100E90009B01AC01BD01CF010895A29FB001B39F9A
:100EA000C001A39F700D811D1124911DB29F700D73
:0C0EB000811D1124911D0895F894FFCFBE
:0C0EBC0007EE82DCD6B2767EC2FEF600A5
:00000001FF
